:020000040800F2
:1000000000070020F1010008E125000899250008FB
:10001000C125000899250008B9250008F30100084A
:10002000F3010008F3010008F3010008C1350008DE
:10003000F3010008F3010008F3010008F3010008D0
:10004000F3010008F3010008F3010008F3010008C0
:10005000F3010008F3010008B5380008DD38000896
:10006000053900082D39000855390008F30100084A
:10007000F3010008F3010008F3010008F301000890
:10008000F3010008F3010008F3010008F301000880
:10009000F301000879250008892500087D3900084A
:1000A000F3010008F3010008F3010008F301000860
:1000B000513A0008F3010008F3010008F3010008B9
:1000C000F3010008F3010008F3010008F301000840
:1000D000F3010008F3010008F3010008F301000830
:1000E000E1390008F3010008F3010008F3010008FA
:1000F000F3010008F3010008F3010008F301000810
:10010000F3010008F3010008F3010008F3010008FF
:10011000F3010008F3010008F3010008F3010008EF
:10012000F3010008F3010008F3010008F3010008DF
:10013000F3010008F3010008F3010008F3010008CF
:10014000F3010008F3010008F3010008F3010008BF
:10015000F3010008F3010008F3010008F3010008AF
:10016000F3010008F3010008F3010008F30100089F
:10017000F3010008F3010008F3010008F30100088F
:10018000F3010008F3010008F3010008F30100087F
:10019000F3010008F3010008F3010008F30100086F
:1001A000F3010008F3010008F3010008F30100085F
:1001B000F3010008F3010008F3010008F30100084F
:1001C000F3010008F3010008F3010008F30100083F
:1001D000F3010008F3010008F3010008F30100082F
:1001E000610F000800000000000000000000000097
:1001F00002E000F000F8FEE772B6374880F30888A6
:10020000364880F3098836483649086040F20000D5
:10021000CCF200004EF63471CEF200010860BFF35C
:100220004F8FBFF36F8F40F20000C0F2F0004EF628
:100230008851CEF200010860BFF34F8FBFF36F8F7C
:100240004FF00000E1EE100A4EF63C71CEF20001D4
:100250000860062080F31488BFF36F8F04F092F8D3
:1002600004F072F94FF055301F491B4A91423CBFD0
:1002700041F8040BFAE71D49184A91423CBF41F886
:10028000040BFAE71A491B4A1B4B9A423EBF51F82E
:10029000040B42F8040BF8E700201849184A914271
:1002A0003CBF41F8040BFAE704F070F804F092F94F
:1002B000144C154DAC4203DA54F8041B8847F9E797
:1002C00000F042F8114C124DAC4203DA54F8041B12
:1002D0008847F9E704F058B8000700200023002001
:1002E0000000000808ED00E00001002000070020E9
:1002F0007048000800230020A4230020A823002029
:1003000044510020E0010008E4010008E401000875
:10031000E40100082DE9F04F2DED108AC1F80CD052
:10032000C3689D46BDEC108ABDE8F08F002383F3BF
:1003300011882846A047002003F0C8FCFEE703F020
:1003400051FC00DFFEE70000F8B500F01BFE03F0F3
:10035000BBFF074604F00CF80546C0BB294B9F4283
:1003600035D001339F4235D0274B27F0FF029A4208
:1003700033D1F8B200F03EFC2E4642F2107400F089
:100380003FFC08B10024264601F0B2F848B3032030
:1003900000F03EF80024264635B11C4B9F4203D0A6
:1003A00003F0DEFF00242646002003F097FF0EB185
:1003B00000F044F800F056FC02F01AF90546C4B902
:1003C00000F098FC4FF47A7003F086FCF7E72E46B5
:1003D0000024D4E704460126D1E7064640F6C414BB
:1003E000CDE740F6C4139C4204BF4FF47A74012653
:1003F000D2E702F0FDF8431BA342E1D900F01EF85A
:10040000DAE700BF010007B0000008B0263A09B0E3
:10041000084B187003280CD8DFE800F00805020824
:10042000022000F00BBE022000F000BE024B0022B2
:100430005A607047A8230020AC23002010B501F0BB
:1004400057F830B1234B03221A70234B00225A6015
:1004500010BD224B224A1C4619680131F8D00433E2
:100460009342F9D16268A242F2D31E4B9B6803F11A
:10047000006303F510439A42EAD203F043FF03F00E
:1004800055FF002000F098FD0220FFF7C1FF164B3A
:100490009A6D00229A65996F9A67996FD96DDA659E
:1004A000D96FDA67D96F196E1A66D3F88010C3F85E
:1004B0008020D3F8803072B64FF0E0233021C3F8AB
:1004C000084DD4E9003281F311889D4683F30888F2
:1004D0001047BDE7A8230020AC23002000900008AF
:1004E000209000080023002000100240094A1368F1
:1004F00049F2690099B21B0C00FB01331360064BF3
:10050000186844F2506182B2000C01FB02001860CE
:1005100080B27047142300201023002010B5002162
:100520001022044600F0A4FD034B03CB2060616061
:100530001868A06010BD00BF9075FF1F2DE9F04145
:10054000ADF5507D0DF13C086EAC40F275120746DA
:100550000D4610A80021C8F8001000F089FD4FF4E6
:10056000C4720021204600F083FD02F041F8254BC3
:100570004FF47A72B0FBF2F0186093E807000223A0
:1005800084E807000DF5ED702382FFF7C7FF4BF2FB
:1005900014531D49238406A804F084F8202384F80A
:1005A00032310DF2EB2606AB0DF1380C1A4603CAB8
:1005B000624530607160134606F10806F6D1414687
:1005C0000122204600F0A0FD00230393AB7E02939E
:1005D00005F11903019380B20123CDE90480009352
:1005E000E97E06A3D3E90023384602F0BFFB0DF5F0
:1005F000507DBDE8F08100BFAFF300809E6AC4214A
:10060000818A46EEB4230020B44600082DE9F0416B
:100610002C4C237ADAB080460D465BBB27A92846CE
:1006200000F082FE0746002842D19DF89D60C82E4A
:100630003ED801464FF4A662204600F019FD4FF463
:100640008073C4F8F8314FF40073C4F80C334FF4DE
:100650004073C4F8203432460DF19E0104F10900C4
:1006600000F0F4FC26449DF89C30777223720BB99D
:10067000EB7E23728122002106AC27A800F0F8FC53
:100680000122214627A800F08BFE00230393AB7EB6
:10069000029305F1190380B201932823CDE90440A8
:1006A0000093E97E05A3D3E90023404602F05EFBF8
:1006B0005AB0BDE8F08100BFAFF3008026417272EE
:1006C000DF25D7B7C0480020F0B5254E4FF48A7516
:1006D00005FB0065F1B096F8D83085F8DC300024D1
:1006E000D822214685F8E8403AA800F0C1FC06F17E
:1006F000090000F0B5FCD5F8E4308DF8F000C2B286
:1007000006AF06F109010DF1F100CDE93A3400F030
:100710009DFC394601223AA800F06EFE80B2CDE978
:10072000047008230127CDE9023706F1D8030193AD
:1007300030230093317A0B4807A3D3E9002302F05A
:1007400015FBA04206DD01F053FFC5F8E000384676
:1007500071B0F0BD2046FBE778F6339F93CACD8D8C
:10076000C0480020CC3300202DE9F0411D4D1E4E25
:100770001E4F86B0284602F025FB034658B30024DE
:10078000CDE90344ADF81440027B8DF8142099683C
:100790004068029403AA03C21B68DFF8548043F048
:1007A0000043029301F026FF821941F100030094F7
:1007B00002A9384601F0B0F8A04205DD284602F053
:1007C00005FB88F80040D5E798F80030072B05D8DE
:1007D000013388F8003006B0BDE8F081014802F02E
:1007E000F5FAF8E7CC33002040420F000034002037
:1007F000F54D002070B50D4614461E4602F012FA63
:1008000050B9022E10D1012C0ED112A3D3E900232E
:10081000C5E90023012007E0282C10D005D8012CC1
:1008200009D0052C0FD0002070BD302CFBD10BA3BC
:10083000D3E90023ECE70BA3D3E90023E8E70BA3FC
:10084000D3E90023E4E70BA3D3E90023E0E700BFEB
:10085000AFF30080401DA12026812A0B78F6339F3C
:1008600093CACD8D9E6AC421818A46EE264172725A
:10087000DF25D7B7F017304A39059E5638B50546FB
:100880000E4C0021013500F0B9FBA4F82C55B4F84A
:100890002C0500F09BFB78B1B4F82C0500F0A6FB0A
:1008A000014648B9B4F82C0500F0A8FBB4F82C3583
:1008B0000133A4F82C35EAE738BD00BFC04800205A
:1008C00010B50A4B0A4A1A6003F5805393F8482082
:1008D0003AB95C6C2CB1204600F088FE204603F04B
:1008E00097FEBDE81040034800F080BE00340020B1
:1008F00008470008304400202DE9F04F8FB000AFCA
:1009000005460C4602F08EF9002849D1237E022BC1
:100910001BD1E38A012B18D101F06AFE0646FFF7CE
:10092000E5FD03464FF4C870DFF8C482B3FBF0F274
:1009300006F5167602FB103316FA83F3C8F800307A
:10094000E37E33B9A34B00221A703C37BD46BDE8A5
:10095000F08F07F12401204600F0A4FC0028F4D118
:1009600007F11400FFF7DAFD97F8264007F11401AC
:10097000224607F1270003F063FE0028E2D10F2C86
:1009800008D8944B1C70D8F80030A3F51673C8F83B
:100990000030DAE797F82410284602F03BF9D4E754
:1009A000E38A282B2BD010D8012B23D0052BCCD1B8
:1009B000BFF34F8F8849894BCA6802F4E062134342
:1009C000CB60BFF34F8F00BFFDE7302BBDD1844E0E
:1009D000E17E327A9142B8D1607E3146002291F8B0
:1009E000DC50854200F0A5800132042A01F58A71AD
:1009F000F5D1AAE721462846FFF7A0FDA5E7214645
:100A00002846FFF703FEA0E7B2F8EC507B6005F143
:100A100003094FEA99094FEA8902D11DC908A8EBD9
:100A2000C1039D46EB460021584600F021FB04F12E
:100A3000EE012A463144584600F008FB7B6813B9A2
:100A4000012000F0B9FA96F8D20000F0BFFA04468F
:100A500030B9307200F0DAFA204600F0ADFAB1E0B9
:100A6000D6F8D4203AB996F8D200B6F82C258242AE
:100A700001D8FFF703FFD6F8D4202A44944208D2C5
:100A800096F8D200B6F82C250130824201D8FFF743
:100A9000F5FE70685FFA89F2594600F0F1FA08B97C
:100AA000C54679E0726896F8D2002A447260D6F89A
:100AB000D42005EB0209C6F8D49000F087FA8145EE
:100AC00009D396F8D220D6F8D4000132001B86F85C
:100AD000D220C6F8D400FF2D0FD80024347200F0C5
:100AE00095FA204600F068FA00F002FD3D4B1881AF
:100AF00008B9FFF7A3FCC54627E7BB6896F8D900FD
:100B00000AFB0362FB68D2F8E41082F8E83001F5D2
:100B10008061C2F8E030C2F8E410FFF7D5FDFFF7BE
:100B200023FE96F8D920013202F0030286F8D9207C
:100B3000B6E74FF48A7A0AFB02F505F1EA0131447F
:100B4000204600F085FCF86000287FF4FEAE3544B6
:100B5000012285F8E82001F04BFDD5F8E020D6ED24
:100B6000007ADFED216A801A192838BF192040F673
:100B7000B832904228BF1046B8EE677A07EE900A66
:100B8000F8EEE77A67EEA67ADFED186AE7EE267AE6
:100B9000FCEEE77AC6ED007A96F8D930BB60BA6809
:100BA00073680AFB02F4321992F8E81059B1D2F8CE
:100BB000E4108B42E8463FF427AF002182F8E810AA
:100BC000C2F8E010C5467368064A9B0A01331381D8
:100BD000BBE600BFC533002000ED00E00400FA05CD
:100BE000C0480020B4230020CDCCCC3D6666663FD3
:100BF000C8330020014B1870704700BFC02300208D
:100C000038B54FF00054134B22689A4220D1124B52
:100C1000627D12481A70237D03724FF48073C0F80E
:100C2000F8314FF40073C0F80C3300254FF44073D3
:100C3000C0F820340A49C0F8E450C922093000F055
:100C400005FAE0222946204600F012FA012038BDBC
:100C50000020FCE79AAD44C5C0230020C048002016
:100C60001600002037B500F043FC194D19492881C2
:100C700002236B7100220123174801F097F800232B
:100C80000193164B164900931648174B4FF48052A8
:100C900001F098FF154B197811B1124801F0BAFF15
:100CA00001F0A6FC0446FFF721FC4FF4C873B0FB2B
:100CB000F3F202FB130304F5167010FA83F00C4BE9
:100CC000186003F055FB08B10F232B8103B030BD32
:100CD000B423002040420F0000340020F507000834
:100CE000C4230020CC330020F9080008C0230020D2
:100CF000C83300202DE9F04F2DED028B90A7D7E9E6
:100D000000670FF24429D9E90089884C95B00DADF0
:100D10009FED848BFFF728FDDFF834B200230C939E
:100D2000ADF83C300D936B6000230DF125028DED85
:100D3000008B4FF0010A09A958468DF825308DF82F
:100D400024A001F0BDFB9DF824200023002A40F0E0
:100D5000AF80204601F066FF0546002847D1DFF846
:100D6000F4B101F045FCDBF8003098423FD301F0CC
:100D70003FFC0790FFF7BAFB079A4FF4C873B0FB2C
:100D8000F3F101FB130302F5167010FA83F0CBF8B0
:100D90000000DFF8C4B19BF800100791002914BFD0
:100DA0002B46534610A88DF83030FFF7B7FB079954
:100DB000C1F11002D2B2062A10AB28BF0622194494
:100DC0000DF13100079200F041F9079A0CAB039343
:100DD000182302930132564BD2B2CDE900A30492FC
:100DE0003B463246204601F063FF8BF8005001F08D
:100DF000FFFB504A504D1368C31AB3F57A7F32D3C4
:100E0000106001F0F7FB02460B46204601F0E8FFB8
:100E1000204601F007FF30B32B7ADFF840A1002B0A
:100E200014BF032302238AF8053001F0E1FB0DF122
:100E3000400B4FF47A730122B0FBF3F05946CAF825
:100E40000000504600F006FA182302933B4B019332
:100E500080B240F25513CDE903B0009342464B46B1
:100E6000204601F025FF2B7AB3B101F0C1FB4FF012
:100E7000000A83464FF48A7295F8D900504400F076
:100E8000030002FB005393F8E810002934D00AF164
:100E9000010ABAF1040FEFD1C82002F01DFF2B7A2E
:100EA000002B7FF434AF15B0BDEC028BBDE8F08FA2
:100EB0004FF0904110A84A6982F010024A61194629
:100EC000102200F0D5F80DF126030AAA0CA9584605
:100ED00000F016FE95E8030011AB83E803009DF8CF
:100EE0003C308DF84C300C9B109310A9DDE90A239F
:100EF000204602F049F917E7D3F8E01049B12B6812
:100F0000FA2B38BFFA23ABEB01010533B1EB430FEA
:100F1000BDD3FFF7D9FB4FF48A720028B7D1BBE7E6
:100F2000AFF300800000000000000000CC33002080
:100F3000C4330020F04D0020C0480020F44D0020B4
:100F4000401DA12026812A0BF1C6A7C1D068080F39
:100F500000340020C8330020C5330020B423002013
:100F600008B5054800F072FEBDE80840034A044990
:100F7000002003F047BB00BF00340020304E0020AB
:100F8000C108000870B503F043F8094E094D3080E0
:100F9000002428683388834208D903F035F82B6889
:100FA00004440133B4F5104F2B60F2D370BD00BF81
:100FB000244E0020F84D002003F0DCB800F1006062
:100FC000920000F5104003F05FB80000054B1A686E
:100FD000054B1B889B1A834202D9104403F014B8B6
:100FE00000207047F84D0020244E0020024B1B6863
:100FF000184403F00FB800BFF84D0020024B1B68E7
:10100000184403F019B800BFF84D0020064991F8C4
:10101000243033B10023086A81F824300822FFF716
:10102000CDBF0120704700BFFC4D0020022802BF49
:101030004FF0904310229A6170470000022802BFCF
:101040004FF090434FF480129A61704710B500231F
:10105000934203D0CC5CC4540133F9E710BD0000C7
:1010600003460246D01A12F9011B0029FAD1704733
:1010700002440346934202D003F8011BFAE770478B
:101080002DE9F8431F4D144695F82420074688465D
:1010900052BBDFF870909CB395F824302BB9202216
:1010A000FF2148462F62FFF7E3FF95F82400C0F1C7
:1010B0000802A24228BF2246D6B24146920005EB62
:1010C0008000FFF7C3FF95F82430A41B1E44F6B23E
:1010D000082E17449044E4B285F82460DBD1FFF772
:1010E00095FF0028D7D108E02B6A03EB82038342E7
:1010F000CFD0FFF78BFF0028CBD10020BDE8F883CD
:101100000120FBE7FC4D00202DE9F0470D46044689
:1011100000219046284640F27912FFF7A9FF2346A6
:1011200020220021284601F0D1FF231D0222202188
:10113000284601F0CBFF631D03222221284601F03F
:10114000C5FFA31D03222521284601F0BFFF04F19E
:10115000080310222821284601F0B8FF04F11003EB
:1011600008223821284601F0B1FF04F111030822BA
:101170004021284601F0AAFF04F112030822482169
:10118000284601F0A3FF04F1140320225021284631
:1011900001F09CFF04F1180340227021284601F061
:1011A00095FF04F120030822B021284601F08EFFAC
:1011B00004F121030822B821284601F087FF04F139
:1011C0002207C0263B46314608222846083601F051
:1011D0007DFFB6F5A07F07F10107F3D104F13203DB
:1011E00008223146284601F071FF002704F1330A36
:1011F00094F832304FEAC7099F4209F5A47615D317
:10120000B8F1000F08D1314604F59973072228463A
:1012100001F05CFF09F24F16274694F832213B1B80
:1012200093420CD3F01DC008BDE8F0870AEB07031A
:1012300008223146284601F049FF0137D8E707F276
:10124000331331460822284601F040FF08360137A3
:10125000E3E7000013B50446084600210160234679
:10126000C0F803102022019001F030FF0198231DE7
:101270000222202101F02AFF0198631D032222216E
:1012800001F024FF0198A31D0322252101F01EFF78
:10129000019804F108031022282101F017FF07200C
:1012A00002B010BDF7B50023047F00910E4607225F
:1012B0001946054601F0CEFD731C00930122002360
:1012C0000721284601F0C6FDC4B9B31C00930522CE
:1012D00023460821284601F0BDFD0D243746B2788B
:1012E000BB1B934211D32B7FA88A0734E408BBB9F8
:1012F000844294BF0020012003B0F0BDAB8ADB0024
:10130000083BDB08B3700824E8E7FB1C0093214688
:1013100000230822284601F09DFD08340137DEE74E
:10132000201A18BF0120E7E7F7B50023047F0091DA
:101330000E4608221946054601F08CFD731CC4B9FF
:101340000822009311462346284601F083FD10240D
:10135000012372785F1C013B934211D32B7FA88A33
:101360000734E408BBB9844294BF0020012003B0D5
:10137000F0BDAB8ADB00083BDB0873700824E7E7AD
:10138000F3190093214600230822284601F062FD4C
:1013900008343B46DDE7201A18BF0120E7E70000CC
:1013A000F8B50E4605461446002181223046FFF767
:1013B0005FFE2B4608220021304601F087FE7CB9F3
:1013C0006B1C07220821304601F080FE0F24012308
:1013D0006A785F1C013B934204D3E01DC008F8BD4E
:1013E0000824F4E7EB1921460822304601F06EFE8E
:1013F00008343B46ECE70000F8B50E4605461446B7
:101400000021CE223046FFF733FE2B462822002152
:10141000304601F05BFE7CB905F108030822282163
:10142000304601F053FE30242F462A7A7B1B93422C
:1014300004D3E01DC008F8BD2824F5E707F109032F
:1014400021460822304601F041FE08340137ECE71E
:10145000F7B5047F00910E460123102200210546B6
:1014600001F0F8FCC4B9B31C0093092223461021F3
:10147000284601F0EFFC192437467288BB1B9A42BC
:1014800011D82B7FA88A0734E408BBB9844294BFE3
:101490000020012003B0F0BDAB8ADB00103BDB086D
:1014A00073801024E8E73B1D0093214600230822A7
:1014B000284601F0CFFC08340137DEE7201A18BFB8
:1014C0000120E7E730B5094D0A4491420DD011F8EB
:1014D000013B5840082340F30004013B2C4013F02B
:1014E000FF0384EA5000F6D1EFE730BD2083B8ED6A
:1014F000F7B5384A106851686B4603C36A463649E7
:101500003648082303F0ACF80446002833D10A25F6
:10151000334A106851686B4603C36A4631492F4805
:10152000082303F09DF80446002849D00369B3F569
:101530005C3F45D8B0F8661041F2B54291423FD1C8
:10154000294A024402F15C018B4239D35C3B2349B6
:1015500000209E1AFFF7B6FF3246074604F16401E9
:101560000020FFF7AFFFA3689F4229D1E3689842AC
:1015700008BF002524E00369B3F55C3F27D8418B01
:1015800041F2B542914220D1174A024402F11001C2
:101590008B4218D3103B114900209D1AFFF792FF90
:1015A0002A46064604F118010020FFF78BFFA368C6
:1015B0009E4202D1E368984201D00D25A8E700259C
:1015C000284603B0F0BD1025A2E70C25A0E70B25A7
:1015D0009EE700BFD8460008DC6F030000900008BB
:1015E000E1460008906F03000870FFF710B5037C18
:1015F000044613B9006803F01BF8204610BD000034
:101600000023BFF35B8FC360BFF35B8FBFF35B8FC0
:101610008360BFF35B8F7047BFF35B8F0068BFF3DE
:101620005B8F704770B505460C30FFF7F5FF05F18D
:10163000080604463046FFF7EFFFA04206D93046C1
:101640006D68FFF7E9FF2544281A70BD3046FFF7A3
:10165000E3FF201AF9E7000070B50546406898B12D
:1016600005F10800FFF7D8FF05F10C0604463046E7
:10167000FFF7D2FF8442304694BF6D680025FFF724
:10168000CBFF013C2C44201A70BD000038B50C463D
:101690000546FFF7C7FFA04210D305F10800FFF78A
:1016A000BBFF04446868B4FBF0F100FB1144BFF3D6
:1016B0005B8F0120AC60BFF35B8F38BD0020FCE77F
:1016C0002DE9F041144607460D46FFF7C5FF844259
:1016D00028BF0446D4B1B84658F80C6B4046FFF713
:1016E0009BFF3044286040467E68FFF795FF331A21
:1016F0009C4203D86C600120BDE8F0816B60A41BA4
:101700003B68AB602044E8600220F5E72046F3E741
:1017100038B50C460546FFF79FFFA04210D305F1F0
:101720000C00FFF779FF04446868B4FBF0F100FB9C
:101730001144BFF35B8F0120EC60BFF35B8F38BDBA
:101740000020FCE72DE9FF41884669460746FFF780
:10175000B7FF6C4606B204EBC6060025B44209D0BA
:101760006268206808EB0501FFF770FC63680834C5
:101770001D44F3E729463846FFF7CAFF284604B060
:10178000BDE8F081F8B505460C300F46FFF744FF81
:1017900005F1080604463046FFF73EFFA0423046FA
:1017A00088BF6C68FFF738FF201A386020B13046D8
:1017B0002C68FFF731FF2044F8BD000073B51446D4
:1017C00006460D46FFF72EFF844228BF04460190CF
:1017D000DCB101A93046FFF7D5FF019B33B9326870
:1017E000C5E90233C5E9002401200CE09C4238BF62
:1017F00001942860019868608442F5D93368AB6031
:10180000241AEC60022002B070BD2046FBE7000005
:101810002DE9FF410F466946FFF7D0FF6C4600B245
:1018200004EBC0050026AC4209D0D4F8048054F87B
:10183000081BB8194246FFF709FC4644F3E7304657
:1018400004B0BDE8F081000038B50546FFF7E0FFC1
:10185000044601462846FFF719FF204638BD000020
:101860007047000010B41346026814680022A446B2
:101870005DF8044B6047000000F5805090F8590473
:101880007047000000F5805090F852047047000047
:1018900000F5805090F958047047000050207047C0
:1018A000302383F3118800F58052D2F89C34D2F8AB
:1018B00098041844D2F894341844D2F87C3418446C
:1018C000D2F88C341844D2F888341844002383F3B7
:1018D0001188704700F58050C0F8541401207047FB
:1018E00038B5C26A936923F001039361044600F09E
:1018F0007FFE0546E36A9B69DB0706D500F078FEAC
:10190000431BFA2BF6D9002004E004F58054012093
:1019100084F8520438BD00002DE9F04F0C4600F564
:10192000805185B01F4691F85234BDF83890054675
:1019300090469BB1D1F878340133C1F878342368EC
:10194000980006D4237B082B0BD9627B0AB10F2B9E
:1019500007D9D1F87C340133C1F87C344FF0FF3023
:1019600010E0302383F31188EB6AD3F8C42012F41B
:10197000001B0AD0D1F880340133C1F88034002034
:1019800080F3118805B0BDE8F08FD3F8C43020682B
:10199000C3F3014A6B6A4822002812FB0A33B4BF22
:1019A00040F08040800418602268520044BF40F03C
:1019B00000501860207B4FEA0A6242EA00425A60F7
:1019C000607B4FEA4A1610B342F440125A60D1F8D5
:1019D000B0240132C1F8B024AA1902F58352117B58
:1019E00041F020011173207B039300F05DFE039B07
:1019F000033080105FFA8BF282420BF1010B0DDA9B
:101A000004EB820103EB820249689160F2E7AA19B4
:101A100002F58352117B60F34511E3E7EB6A012283
:101A200002FA0AF2C3F8CC2005EB4A11AB1903F510
:101A3000825301F58251C3E904871831234604F12A
:101A40000C0253F8040B41F8040B9342F9D11B88A4
:101A50000B802E4441F2680346F803A006F5805639
:101A600009F0030396F86C2043F0100322F01F02E4
:101A7000134386F86C30002383F31188CDF800906F
:101A800042463B462146284600F0D4FD012079E736
:101A900013B500F580540191606CFFF7DDFD1F2840
:101AA0000AD90199606C2022FFF74CFEA0F12003B7
:101AB0005842584102B010BD0020FBE708B5302362
:101AC00083F3118800F58050406CFFF799FD0023E7
:101AD00083F3118808BD0000002202608281426009
:101AE0008260704710B500220023C0E90023002364
:101AF000044603810C30FFF7EFFF204610BD0000C5
:101B00002DE9F0479A4688B007468846914630232B
:101B100083F3118807F580546846FFF7E3FF606C94
:101B2000FFF780FD1F282DD9606C20226946FFF742
:101B30008BFE202826D194F852341BB303AD4446C3
:101B400005AB2E4603CE9E4220606160354604F10F
:101B50000804F6D130682060B388A380DDE9002353
:101B6000C9E90023BDF80830AAF80030002383F348
:101B7000118853464A464146384608B0BDE8F0470A
:101B800000F046BD002080F3118808B0BDE8F08762
:101B90002DE9F84F00230646C0E90133284B46F8EB
:101BA000303B00F5815405468846374610343846A8
:101BB0002037FFF797FFA742F9D105F580544FF47E
:101BC000805326630026C4E90D366764012305F5BA
:101BD000835705F5A359E66384F8403084F848300C
:101BE000103709F110094FF0000A4FF0000B47E9D8
:101BF00008ABA7F11800FFF76FFF203747F8286CF4
:101C00004F45F4D184F85884A4F85A64A4F85C646D
:101C1000A4F85E6484F86064A4F86264A4F8646460
:101C2000A4F8666484F86864B8F1000F02D005482F
:101C300000F0D8FC044BEB622846BDE8F88F00BFEB
:101C400008470008EC4600080064004010B5044B4B
:101C5000197804464A1C1A70FFF79AFF204610BDF7
:101C60002D4E00202DE9F84315460C4600295CD086
:101C7000022001F019FE2E49B0FBF4F78C428CBF14
:101C80000A2111214B1EB7FBF1F601FB1671DAB2E6
:101C900021B1022B1946F5D8002032E0731EB3F5AE
:101CA000806FF9D2C2EBC20808F103014FEAE10EDE
:101CB000C1F3C701A2EB010C0EF101094FF47A73D5
:101CC0005FFA8CF70EFB033E59FA8CFCBEFBFCFC62
:101CD000BCF5617F17DC1FFA8CF34A1C57FA82F2BD
:101CE0007243B0FBF2F08442D6D14A1E0F2AD3D8F9
:101CF0007A1E072AD0D801202B806E802871697146
:101D0000AF71BDE8F88308F1FF314FEAE10CC1F390
:101D1000C701521A0CF1010ED7B20CFB03335EFA65
:101D200082F2B3FBF2F39BB2D7E70846E9E700BFC4
:101D30003F420F0030B50D4B0D4D05201C786C4314
:101D40008C420ED15978518099785171D97891711E
:101D5000197911715B7903EB83035B001380012018
:101D600030BD013803F10603E8D1F9E74847000820
:101D700040420F000B4B10B54FF454720446002143
:101D80001846FFF775F9084BA3614033E361D83378
:101D90002362F0336362E36A60610022C3F8C0200B
:101DA00010BD00BF00A4004070A400402DE9F04F1A
:101DB00000F580551F4695F85834012B89B004462C
:101DC0008946904604D90026304609B0BDE8F08F18
:101DD0009A4A52F8231009B942F823009848C4F8E7
:101DE0000C900178277499B9302383F31188954BAF
:101DF0009A6D42F000729A659A6B42F000729A6393
:101E00009A6B22F000729A630123037081F31188A8
:101E100095F851647EB9302383F31188032115208E
:101E200001F056FE0321162001F052FE012385F831
:101E3000513486F31188302383F31188E26A936961
:101E400023F01003936100F0D3FB8246E36A9E699E
:101E500016F0080609D000F0CBFBA0EB0A03FA2B22
:101E6000F4D9002686F31188AEE79A6942F00102A0
:101E70009A6100F0BDFB8246E36A9A69D00706D4F6
:101E800000F0B6FBA0EB0A03FA2BF5D9E9E79A6953
:101E900042F002029A61E36A4FF0000AC3F854A0CC
:101EA0008AF31188686CFFF7ABFB04F5825B0BF1DA
:101EB000100B202200216846FFF7DAF802A8FFF78E
:101EC0000BFECDF818A06A460BEB06030DF1180EB9
:101ED0009446BCE80300F44518605960624603F17B
:101EE0000803F5D1DCF80000186020369CF80420C7
:101EF0001A71B6F5806FDCD1002304F5A25285F883
:101F0000503485F853341A3249462046FFF7AAFE6A
:101F1000064690B9E26A936923F00103936100F0E9
:101F200067FB0546E36A9B69D9077FF54CAF00F074
:101F30005FFB431BFA2BF5D945E795F85E34C5F8EE
:101F40006C94591E95F85F34E26A013B1B0243EA28
:101F5000416395F8601401390B43B5F85C140139FD
:101F600043EA0143D361B8F1000F36D004F5A35220
:101F7000023241462046FFF7DDFE90B9E26A9369DE
:101F800023F00103936100F033FB0546E36A9B698C
:101F9000DA077FF518AF00F02BFB431BFA2BF5D9BE
:101FA00011E795F86724C5F87084511E95F86824E8
:101FB000E36A013A120142EA012295F866140139F6
:101FC0000A43B5F86414013942EA014242F40002BE
:101FD000DA60E36A4FF420629A642046FFF7CAFE93
:101FE000002385F85934E36A6FF040421A65E36ACA
:101FF000154A5A65E36A44229A65E36A0722C3F8E0
:10200000DC20E36A03229742DA653FF4DDAEE26A40
:10201000936923F00103936100F0EAFA0746E36A4B
:102020009B69DB0705D500F0E3FAC31BFA2BF6D951
:10203000C9E6012385F85234C6E600BF284E0020C9
:102040002C4E0020001002409B0008002DE9F04FAC
:10205000054689B090469946002741F2680A00F586
:102060008056EB6AD3F8D430FB40D80751D505EB46
:10207000471252444FEA471B1379190749D4D6F83F
:1020800084340133C6F8843405F5A553C3E90089C7
:1020900013799A0648BFD6F8B43405EB0B0248BF53
:1020A0000133524448BFC6F8B434137943F00803EF
:1020B0001371DB0722D596F85334FBB105F5825432
:1020C000183468465C44FFF70DFD03AB04F1080CBF
:1020D000206861681A4603C2083464451346F7D184
:1020E00020681060A2889A800123ADF808302B6820
:1020F000CDE90089DB6B694628469847D6F8A834B5
:10210000D6F854040133C6F8A83410B103681B692B
:1021100098470137202FA4D109B0BDE8F08F000007
:102120002DE9F04F8DB004460F4600F063FA824669
:102130008946002F56D1E36AD3F89020920141BF1F
:1021400004F58051D1F898240132C1F89824D3F8CD
:102150009020160703D100200DB0BDE8F08FD3F812
:102160009050E669C5F30125482303FB0566E84660
:102170004046FFF7B1FC326851004ABF22F060438D
:10218000C2F38A4343F00043920048BF43F08043C8
:102190000093736813F400131FBF04F580520123EA
:1021A0008DF80D30D2F8B8340EBF8DF80D300133F4
:1021B000C2F8B834F38803F00F038DF80C304FF0F9
:1021C000000B9DF80C0000F06FFA5FFA8BF3984259
:1021D00020D9F2180CA90B44127A03F82C2C0BF11D
:1021E000010BEEE7012FB6D1E36AD3F898209501F1
:1021F00041BF04F58051D1F898240132C1F89824E8
:10220000D3F898201007A6D0D3F89850266AC5F3C3
:102210000125A9E7EFB9E36AC3F8945004A8FFF7D2
:1022200061FC98E80F0007AD07C52B800023ADF8CF
:10223000183023682046CDE904A9DB6B04A9984730
:1022400004F5805458B1D4F890340133C4F8903474
:1022500082E7012F04BFE36AC3F89C50DEE7D4F89D
:1022600094340133C4F89434012075E72DE9F0412A
:1022700005460F4600F58054012639462846FFF7EB
:102280004FFF10B184F85364F7E7D4F8A834D4F8BA
:1022900054040133C4F8A83420B10368BDE8F04108
:1022A0001B691847BDE8F081F0B5C36A1A6C12F4D7
:1022B0007F0F2BD000F580541B6CC4F8AC3441F276
:1022C0006805002347194FF0010C00EB43122A4424
:1022D0005E01117911F0020F15D0490713D4B959D5
:1022E000C66AD6F8C8E00CFA01F111EA0E0F0AD05E
:1022F000C6F8D010117941F004011171D4F88C2482
:102300000132C4F88C240133202BDED1F0BD000053
:1023100010B5254C254B226802B338B31A6D12064E
:102320000ED580221A6500F065F950EA01020B46CD
:1023300002D0013861F1000302462068FFF786FEF3
:102340001A4A136D1B032AD523684FF4002103F5A5
:1023500080531165012283F8592420E001221A6577
:1023600008221A654FF480621A6510BD196DC807FE
:1023700002D4196D890705D503211965104600217E
:10238000FFF774FF094B1A6D100702D41A6DD106BE
:1023900005D518221A6520680121FFF767FF20681C
:1023A000BDE81040FFF780BF284E002000640040C9
:1023B00008B5302383F31188FFF776FF002383F3FA
:1023C000118808BDC36AD3F8C40080F40010C0F3BC
:1023D0004050704708B5302383F3118800F58050D2
:1023E000406CFFF71FF9002383F3118843090CBFEA
:1023F0000120002008BD000000F5805393F8592407
:1024000062B1C16A8A6922F001028A61D3F89C2410
:102410000132C3F89C24002283F85924704700003D
:102420002DE9F743302181F3118800F582511031F5
:10243000002541F2680E4FF0010800F5805C00EBCA
:1024400045147444267977071CD4F6061AD5D0F8BB
:102450002C908E69D9F8C87008FA06F63E4211D061
:102460004F6801970F689742019F9F410AD2C9F8B0
:10247000D060267946F004062671DCF888440134E1
:10248000CCF888440135202D01F12001D7D100235B
:1024900083F3118803B0BDE8F0830000F8B51E4651
:1024A000002313700F4605461446FFF793FF80F094
:1024B000010038701EB12846FFF784FF2070F8BD78
:1024C0002DE9F04F85B09946DDE90EA30D46029344
:1024D0001378019391F800B08046164600F08AF810
:1024E0002B7804460F4613B93378002B41D022468F
:1024F0003B464046FFF794FFFFF75AFFFFF77CFF8C
:102500004B4632462946FFF7C9FF2B7833B1BBF162
:10251000000F03D0012005B0BDE8F08F337813B170
:10252000019B002BF6D108F580530393029B544581
:1025300077EB03031DD2039BD3F85404C8B103689F
:10254000AAEB04011B6898474B4632462946404691
:10255000FFF7A4FF2B7813B1BBF1000FDAD133786A
:1025600013B1019B002BD5D100F044F804460F466F
:10257000DCE70020CFE7000008B50020FFF7C8FE29
:10258000BDE8084001F050B808B50120FFF7C0FED3
:10259000BDE8084001F048B800B59BB0EFF30981F1
:1025A00068226846FEF752FDEFF30583014B9B6BF3
:1025B000FEE700BF00ED00E008B5FFF7EDFF00000B
:1025C00000B59BB0EFF3098168226846FEF73EFD37
:1025D000EFF30583014B5B6BFEE700BF00ED00E00E
:1025E000FEE700000FB408B5029801F025FBFEE7F6
:1025F00001F006BE01F0E8BD13B56C4684E80600A4
:10260000031D94E8030083E80500012002B010BD1B
:1026100073B58568019155B11B885B0707D4D0E974
:1026200000369B6B9847019AC1B23046A8470120FB
:1026300002B070BDF0B5866889B005460C465EB143
:10264000BDF838305B070AD4D0E900379B6B984758
:102650002246C1B23846B047012009B0F0BD002281
:102660000023CDE900230023ADF808300A4603AB70
:1026700001F10806106851681C4603C40832B242D2
:102680002346F7D1106820609288A280FFF7B2FF3E
:102690000423ADF808302B68CDE90001DB6B6946F7
:1026A00028469847D8E70000082817D909280CD0F1
:1026B0000A280CD00B280CD00C280CD00D280CD0DC
:1026C0000E2814BF4020302070470C207047102087
:1026D0007047142070471820704720207047000072
:1026E0002DE9F041456A15B94162BDE8F0814B68BA
:1026F00023F06047C3F38A464FEAD37EC3F3807862
:1027000016EA230638BF3E46AC462B465A68BEEB57
:10271000D27F22F060440AD0002A18DAA40CB44216
:1027200017D19D420FD10D60DEE71346EEE7A742B9
:1027300007D102F08044C2F3807242450BD054B1FD
:10274000EFE708D2EDE7CCF800100B60CDE7B4421C
:1027500001D0B442E5D81A689C46002AE5D1196038
:10276000C3E700002DE9F047089D01F007044FEA98
:10277000D508224405F0070500EBD1004FF47F494E
:10278000944201D1BDE8F08704F0070705F0070A7D
:1027900057453E4638BF5646C6F10806111B8E42C5
:1027A00028BF0E46E10808EBD50E415C13F80EC0B9
:1027B000B94029FA06F721FA0AF1FFB28CEA0101C1
:1027C00047FA0AF739408CEA010C03F80EC034448A
:1027D0003544D5E780EA0120082341F2210201B205
:1027E0004000002980B203F1FF33B8BF504013F01E
:1027F000FF03F4D17047000038B50C468D18A54290
:1028000000D138BD14F8011BFFF7E4FFF7E7000023
:1028100042684AB1136843604389818901339BB29E
:102820009942438138BF83811046704770B588B0A4
:10283000202204460D4668460021FEF719FC20467A
:102840000495FFF7E5FF024658B16B46054608AE12
:102850001C4603CCB44228606960234605F1080594
:10286000F6D1104608B070BD082817D909280CD039
:102870000A280CD00B280CD00C280CD00D280CD01A
:102880000E2814BF4020302070470C2070471020C5
:1028900070471420704718207047202070470000B0
:1028A000082817D90C280CD910280CD914280CD9B1
:1028B00018280CD920280CD930288CBF0F200E20C6
:1028C0007047092070470A2070470B2070470C2082
:1028D00070470D20704700002DE9F843078C072F43
:1028E00004461ED9D0E9029800254FF6FF73C5F1C2
:1028F0002006A5F1200029FA05F108FA06F628FAC3
:1029000000F031430143C9B21846FFF763FF0835B1
:10291000402D0346EBD1E1693A46BDE8F843FFF7A5
:102920006BBF4FF6FF70BDE8F883000010B54B6831
:1029300023B9CA8A63F30902CA8210BD04691A68FE
:102940001C600361C38A013BC3824A60EFE7000059
:102950002DE9F84F1D46CB8A0F46C3F3090105291F
:10296000814692460B4630D00020AAB207F11A04E5
:102970009EB2042E1FFA80F80FD8904503F1010390
:1029800006D3FB8A0A4462F30903FB8201201AE0A2
:102990001AF80060E6540130EAE79045F1D2A1F15F
:1029A000050B1C237C68BBFBF3F203FB12BB1FFA75
:1029B0008BF6002C45D14846FFF72AFF044638B96C
:1029C00078606FF00200BDE8F88F4FF00008E6E78E
:1029D000002606607860ADB24FF0000B454510D977
:1029E0000AEB0803221D13F8011B9155B1B208F13F
:1029F00001081B291FFA88F82BD0454506F101066E
:102A0000F1D8FB8AC3F30902154465F30903BCE757
:102A1000013292B21C462368002BF9D16B1F0B4484
:102A20001C21B3FBF1F301339BB29A42D3D2BBF129
:102A3000000FD0D14846FFF7EBFE20B9C4F800B034
:102A4000BFE70122E7E7C0F800B05E462060044619
:102A5000C1E74545D5D94846FFF7DAFE08B92060F9
:102A6000AFE7C0F800B0002620600446B6E70000DB
:102A70002DE9F04F2DED028B1C4683B05B6901926E
:102A800007468846002B00F09A80238C2BB1E26920
:102A9000002A00F09480072B35D807F10C00FFF7CF
:102AA000B7FE054638B96FF00205284603B0BDEC05
:102AB000028BBDE8F08F14220021FEF7D9FA228C98
:102AC000E16905F10800FEF7C1FA208C013080B2FF
:102AD000FFF7E6FEFFF7C8FE013880B22084013020
:102AE00028746369228C1B782A4403F01F0363F067
:102AF0003F0348F000411372384669602946FFF7EA
:102B0000EFFD0125D1E700F10C034FF0000908EEBD
:102B1000103A4FF0800A4E464D4618EE100AFFF765
:102B200077FE83460028BED014220021FEF7A0FACB
:102B3000002E3AD1019BABF8083002220BF1080EAF
:102B40001FFA82FC0CF10100BCF1060F218C80B24F
:102B500001D88E422BD3FFF7A3FEFFF785FE6269F3
:102B60001278013802F01F028E4208BF4FF0400A6F
:102B700042EA49121BFA80F14AEA020A013048F09F
:102B8000004281F808A08BF81000CBF804205946C9
:102B90003846FFF7A5FD238C0135B3422DB289F0ED
:102BA00001094FF0000AB8D17FE70022C6E7E169CA
:102BB000895D0EF802100136B6B20132C0E76FF03F
:102BC000010572E7F8B515460E463022002104468D
:102BD0001F46FEF74DFA069B6360B5F5001F079B85
:102BE000A76034BF6A094FF6FF72A36297B2E6612D
:102BF00004F1100000239A4206D800230360A78244
:102C0000E3822383E360F8BD06600133304620365B
:102C1000F1E7000003781BB94BB2002BC8BF01706D
:102C20007047000000787047F8B50C46C969074640
:102C300011B9238C002B37D1257E1F2D34D838783D
:102C400028BB228C072A2CD8268A36F003032BD1E6
:102C50004FF6FF70FFF7D0FD20F001003102400475
:102C600041EA0561400C41EA40254FF6FF722346D8
:102C700029463846FFF7FCFE002807DD6269137815
:102C80000133DBB21F2B88BF00231370F8BD218AEC
:102C90002D0645EA012505432046FFF71DFE0246A5
:102CA000E5E76FF00300F1E76FF00100EEE70000E9
:102CB00070B58AB0044616460021282268461D4693
:102CC000FEF7D6F9BDF83830ADF810300F9B0593FC
:102CD0009DF840308DF81830119B07936946BDF878
:102CE0004830ADF820302046CDE90265FFF79CFF63
:102CF0000AB070BD2DE9F041D36905460C46164671
:102D00000BB9138C5BBB377E1F2F28D895F800803A
:102D1000B8F1000F26D03046FFF7DEFD33782102F0
:102D200041EAC33141EA0801338A41EA076141EAD5
:102D300003410246334641F080012846FFF798FEE2
:102D400000280ADD3378012B07D17269137801332B
:102D5000DBB21F2B88BF00231370BDE8F0816FF03A
:102D60000100FAE76FF00300F7E70000F0B58BB061
:102D700004460D4617460021282268461E46FEF7E7
:102D800077F99DF84C305A1E534253418DF800306C
:102D90009DF84030ADF81030119B05939DF84830F8
:102DA0008DF81830149B07936A46BDF85430ADF87F
:102DB000203029462046CDE90276FFF79BFF0BB075
:102DC000F0BD0000406A00B104307047436A1A68E1
:102DD000426202691A600361C38A013BC382704781
:102DE0002DE9F041D0F82080194E14461D46414689
:102DF000002709B9BDE8F081D1E90223A21A65EBE9
:102E00000303964277EB03031ED2036A8B420DD174
:102E1000FFF78CFD036A1B68036203690B60C38ABA
:102E20000161016A013BC3828846E2E7FFF77EFD4C
:102E30000B68C8F8003003690B60C38A0161013B6D
:102E4000C382D8F80010D4E788460968D1E700BFEC
:102E500080841E002DE9F04F8BB00D46DDF85090B8
:102E600014469B468046002800F01981B9F1000FF6
:102E700000F01581531E3F2B00F21181012A03D16E
:102E8000BBF1000F40F00B810023CDE90833B8F807
:102E90001430B5EBC30F4FEAC30703D300200BB0C8
:102EA000BDE8F08F2B199F42D8F80C303ABF7F1B3A
:102EB000FFB227461BB9D8F81030002B7AD0272D47
:102EC0004ED8C5F12806B7424FF000032CBFF6B22A
:102ED0003E4600932946D8F8080008AB3246FFF773
:102EE00041FCA7EB060A35445FFA8AFAB8F81430B9
:102EF00003F10053053BDB000493D8F80C30039337
:102F00002821039B13B1BAF1000F2CD1D8F810007F
:102F100040B1BAF1000F05D0009608AB5246691ACD
:102F2000FFF720FC38B2002FB8D066070AD00AABF2
:102F300003EBD401624211F8083C02F0070213418E
:102F400001F8083C082C3CD9102C40F2B580202C0C
:102F500040F2B780BBF1000F00F09C80082334E002
:102F6000BA460026C2E7049BE02B28BFE023069365
:102F70000B44AB42059314D95A1B03980096924513
:102F800034BF5246D2B2691A08AB04300792FFF739
:102F9000E9FB079A1644AAEB020A1544F6B25FFA57
:102FA0008AFA049B069A05999B1A0493039B1B6853
:102FB0000393A6E70093D8F8080008AB3A462946E1
:102FC000AEE7BBF1000F13D00123B4EBC30F6CD0FD
:102FD000082C12D89DF82030621E23FA02F2D50781
:102FE00006D54FF0FF3202FA04F423438DF8203067
:102FF0009DF8203089F8003051E7102C12D8BDF828
:103000002030621E23FA02F2D10706D54FF0FF32BC
:1030100002FA04F42343ADF82030BDF82030A9F8BB
:1030200000303CE7202C0FD80899631E21FA03F3E7
:10303000DA0705D54FF0FF3202FA04F40C43089486
:10304000089BC9F800302AE7402C2BD0DDE9086541
:10305000611EC4F12102A4F1210326FA01F105FA4F
:1030600002F225FA03F311431943CB0712D50122CB
:10307000A4F12003C4F1200102FA03F322FA01F1C2
:10308000A240524243EA010363EB430332432B4322
:10309000CDE90823DDE90823C9E90023FFE66FF045
:1030A0000100FCE66FF00800F9E6082CA0D9102C0E
:1030B000B3D9202CEED8C3E7BBF1000FADD002236B
:1030C00083E7BBF1000FBBD004237EE730B5012AB4
:1030D000144638BF0124402C85B028BF4024002569
:1030E000012ACDE9025518D81B788DF808306307FE
:1030F0000AD004AB03EBD405624215F8083C02F099
:103100000702934005F8083C00910346224600213F
:1031100002A8FFF727FB05B030BD082AE4D9102A22
:1031200003D81B88ADF80830E1E7202A8DBFD3E92A
:1031300000231B680293CDE90223D8E710B5CB68C2
:103140001BB98B600B618B8210BD04691A681C600F
:103150000361C38A013BC382CA60F0E703064CBF28
:10316000C0F3C0300220704708B50246FFF7F6FFF3
:10317000022806D15306C2F30F2001D100F003004C
:1031800008BDC2F30740FBE72DE9F04F93B0CDE94E
:1031900003230A6804461046FFF7E0FF022814BF25
:1031A000C2F306260026002A0D46824680F2F281EE
:1031B00012F0C04940F0EE81097B002900F0EA815D
:1031C000022803D02378B34240F0E781C2F30463BE
:1031D0000693104602F07F030593FFF7C5FF059B9A
:1031E00029444FEA834848EA0A4848EA4668CE78C4
:1031F00000230022CDE90823F309834648EA0008AA
:10320000029367D0059B009302466768534608A95E
:103210002046B847002800F0C381276A4FB94146CD
:1032200004F10C00FFF702FB074690B96FF00200B3
:1032300054E03B6998450DD03F68002FF9D14146D5
:1032400004F10C00FFF7F2FA07460028EED0236ADB
:103250003B60276297F817C006F01F08CCF3840C78
:10326000ACEB08001FFA80FE0028B8BF0EF120006A
:10327000A8EB0C031FFA83FED7E90221B8BF00B206
:10328000002B0793BEBF0EF120031BB2079352EA37
:10329000010338D0039BDFF824E39A1A049B4FF014
:1032A000000C63EB010196457CEB01032BD36B7B98
:1032B00097F81AE0734519D1029B002B78D00128AA
:1032C00021DC7868F8B9DFF8F0C2944570EB0103AF
:1032D00016D337E0276A27B96FF00C0013B0BDE8AA
:1032E000F08F3B699845B5D03F68F4E7B24890420B
:1032F0007CEB010301D30020F0E7029B002BFAD006
:10330000079B0F2B17DCFA7DB30002F0030203F0DA
:103310007C031343FB7539462046FFF707FB6B7BA5
:10332000BB76029B3BB9FB7DC3F38402013262F39F
:103330008603FB75D0E76A7BBB7E9A42DBD1029B9A
:10334000002B35D0B309022B32D0039BBB60049B0A
:10335000FB60142200210DA8FDF78AFE039B0A934F
:10336000049B0B932B1D0C932B7BADF83EB0013BC4
:10337000DBB2ADF83C30069B8DF84230059B8DF8F2
:10338000433094F82C308DF840A083F001038DF881
:1033900044308DF84180A3680AA920469847FB7DF8
:1033A000C3F38403013303F01F039B02FB82A2E7F4
:1033B000FB7DC6F34012B2EBD31F40F0F480C3F3A1
:1033C0008403434540F0F280029A2B7BB609002A21
:1033D0004DD0F2075DD4032B40F2EB80039BBB6022
:1033E000049BFB602B7BAE1D033BDBB232463946B0
:1033F00004F10C00FFF7ACFA00280CDA394620463D
:10340000FFF794FAFB7DC3F38403013303F01F033A
:103410009B02FB820AE7DDE90884AB883B834FF619
:10342000FF73C9F12000A9F1200228FA09F104FA7A
:1034300000F0014324FA02F211431846C9B2FFF723
:10344000C9F909F10809B9F1400F0346E9D1B88279
:103450002A7B033AD2B23146FFF7CEF9FB7DB88220
:10346000DA43C2F3C01262F3C713FB7543E786B9B0
:103470002E1D013BDBB23246394604F10C00FFF74A
:1034800067FA0028BADB2A7BB88A013AD2B2314601
:10349000E2E7F98AC1F30901013B0429DAB25BD8FA
:1034A000281D002307F11B069A4208D910F801CB0A
:1034B00006F801C0013101330529DBB2F4D10399CB
:1034C0000A9104990B91934207F11B010C9138BFAB
:1034D000043379680D9134BF55FA83F300230E93BA
:1034E000FB8AADF83EB0C3F309031A44069B8DF87E
:1034F0004230059B8DF8433094F82C30ADF83C20D9
:1035000083F001038DF8443000238DF840A08DF83E
:1035100041807B602A7BB88A013A291DFFF76CF94C
:103520003B8BB882834203D1A3680AA920469847FF
:1035300020460AA9FFF702FEFB7DBA8AC3F3840383
:10354000013303F01F039B02FB823B8B9A420CBFAB
:1035500000206FF01000C1E67B68002BAFD0052083
:1035600001E01C3033461E68002EFAD1091A081DEE
:103570002E1D184401EB090CBCF11B0F5FFA89F3F7
:103580009DD89A429BD916F8013B00F8013B09F1FE
:103590000109EFE76FF00900A0E66FF00A009DE671
:1035A0006FF00B009AE66FF00D0097E66FF00E00DB
:1035B00094E66FF00F0091E640420F0080841E00F9
:1035C000EFF3098305494A6B22F001024A6368332D
:1035D00083F30988002383F31188704700EF00E02C
:1035E000302080F3118862B60C4B0D4AD96821F463
:1035F000E0610904090C0A43DA60D3F8FC200949A8
:1036000042F08072C3F8FC200A6842F001020A60AE
:103610002022DA7783F82200704700BF00ED00E037
:103620000003FA05001000E010B5302383F3118881
:103630000E4B5B6813F4006314D0F1EE103AEFF315
:103640000984683C4FF08073E361094BDB6B2366B0
:1036500084F3098800F0BAFA10B1064BA36110BDDB
:10366000054BFBE783F31188F9E700BF00ED00E0AD
:1036700000EF00E03F03000842030008434B4FF413
:10368000007270B51A605A6912F4C06FFBD1404BDA
:103690009A6802F00C02042A20D01A6842F4807260
:1036A0001A601A685205FCD501229A609A6802F0E5
:1036B0000C02042AFAD13749374A0A600A6812F024
:1036C0000F02FBD1C3F8982063221A601A68960390
:1036D000FCD42E4A4FF48071C2F88010C468E50310
:1036E00006D51A6842F480321A601A689103FCD534
:1036F000C269D20709D5D3F8982042F00102C3F875
:103700009820D3F898209607FBD54269DA6044F4F4
:1037100080721A6004F0807111B11A689501FBD5AE
:10372000996802691B4E22F0030501F00301294349
:10373000996085693560316869400907FBD1134993
:1037400005680D6046684E608068C1F880006E04B0
:1037500017D448698505FCD4996802F0030021F06C
:1037600003010143996092009968514011F00C0FD8
:10377000FAD1E2055EBF1A6822F480721A60002056
:1037800070BD48698005FCD5E6E700BF00700040C9
:1037900000100240002002400006040008B500F0BE
:1037A00083F9BDE8084000F05BB9000010B5394C62
:1037B0003948A36A4FF0FF32A262A36A0023A362D2
:1037C000A16AE16A61F07F01E162E16A01F07F01D3
:1037D000E162E16A216B2263216B2363216BA16BA0
:1037E000A263A16BA363A16BE16BE263E16BE36393
:1037F000E16B216C2264226C2364226C226E42F005
:1038000001022266D4F8802022F00102C4F8802050
:10381000D4F88020A26D42F08052A265A26F22F0FF
:103820008052A267A26F1D4A4FF400419160D3609D
:10383000136253629362D362136353639363D363DC
:10384000136453649364D36413655365116841F43E
:1038500080711160D4F8902012F4407F1EBF4FF4A5
:103860008032C4F89020C4F890300D4A0023A36041
:10387000C4F88820C4F89C30FFF700FF10B1094855
:1038800000F0DAF9D4F8903023F00323C4F8903034
:1038900010BD00BF001002407047000800700040DB
:1038A0005501005168470008014B53F8200070474C
:1038B00018230020074A08B5536903F00103536138
:1038C00023B1054A13680BB150689847BDE808401A
:1038D000FFF7AABE00040140C4500020074A08B503
:1038E000536903F00203536123B1054A93680BB196
:1038F000D0689847BDE80840FFF796BE0004014035
:10390000C4500020074A08B5536903F0040353610B
:1039100023B1054A13690BB150699847BDE80840C7
:10392000FFF782BE00040140C4500020074A08B5DA
:10393000536903F00803536123B1054A93690BB13E
:10394000D0699847BDE80840FFF76EBE000401400B
:10395000C4500020074A08B5536903F010035361AF
:1039600023B1054A136A0BB1506A9847BDE8084075
:10397000FFF75ABE00040140C4500020164B10B59A
:103980005C6904F478725A61A30604D5134A936AF9
:103990000BB1D06A9847600604D5104A136B0BB17F
:1039A000506B9847210604D50C4A936B0BB1D06B32
:1039B0009847E20504D5094A136C0BB1506C98473F
:1039C000A30504D5054A936C0BB1D06C9847BDE8AC
:1039D0001040FFF729BE00BF00040140C450002082
:1039E000194B10B55C6904F47C425A61620504D538
:1039F000164A136D0BB1506D9847230504D5134A31
:103A0000936D0BB1D06D9847E00404D50F4A136E47
:103A10000BB1506E9847A10404D50C4A936E0BB1BC
:103A2000D06E9847620404D5084A136F0BB1506FEB
:103A30009847230404D5054A936F0BB1D06F98477C
:103A4000BDE81040FFF7F0BD00040140C450002065
:103A500008B500F0F3FCBDE80840FFF7E5BD000045
:103A6000062108B5084600F033F80621072000F0CB
:103A70002FF80621082000F02BF80621092000F07D
:103A800027F806210A2000F023F80621172000F06D
:103A90001FF80621282000F01BF8BDE80840072188
:103AA0001C2000F015B800004FF0E02300225868F9
:103AB0004FF0FF31930003F1604303F5614301329E
:103AC0009042C3F88010C3F88011F3D27047000011
:103AD00000F1604303F561430901C9B283F80013A3
:103AE000012200F01F039A4043099B0003F1604349
:103AF00003F56143C3F880211A6070470023037502
:103B0000826803691B6899689142FBD25A68036016
:103B10004260106058607047002303758268036933
:103B20001B6899689142FBD85A6803604260106034
:103B30005860704708B50846302383F311880B7D21
:103B4000032B05D0042B0DD02BB983F3118808BDAE
:103B50008B6900221A604FF0FF338361FFF7CEFFBD
:103B60000023F2E7D1E9003213605A60F3E7000066
:103B7000FFF7C4BF054BD9680875186802681A605A
:103B8000536001220275D860FCF7C4BB384E002098
:103B900030B50C4BDD684B1C87B004460FD02B466C
:103BA000094A684600F02AF92046FFF7E3FF009B28
:103BB00013B1684600F02CF9A86907B030BDFFF7D3
:103BC000D9FFF9E7384E0020353B0008044B1A684E
:103BD000DB6890689B68984294BF00200120704782
:103BE000384E0020084B10B51C68D86822681A604F
:103BF000536001222275DC60FFF78EFF01462046EC
:103C0000BDE81040FCF786BB384E002038B5074CA5
:103C100007490848012300252370656000F03CFC3B
:103C20000223237085F3118838BD00BFA050002007
:103C300094470008384E002008B572B6044B18654A
:103C400000F0ACFA00F05CFB024B03221A70FEE7B6
:103C5000384E0020A050002000F010B98B600223E5
:103C600008618B82084670478368A3F1840243F899
:103C7000142C026943F8442C426943F8402C094A49
:103C800043F8242CC26843F8182C022203F80C2CA9
:103C9000002203F80B2C044A43F8102CA3F1200057
:103CA000704700BF2D030008384E002008B5FFF70D
:103CB000DBFFBDE80840FFF75BBF0000024BDB689D
:103CC00098610F20FFF756BF384E0020302383F352
:103CD0001188FFF7F3BF000008B50146302383F3D6
:103CE00011880820FFF754FF002383F3118808BDD3
:103CF00010B503689C68A2420CD85C688A600B60AF
:103D00004C602160596099688A1A9A604FF0FF33BD
:103D1000836010BD1B68121BECE700000A2938BF46
:103D20000A2170B504460D460A26601900F0AEFB64
:103D300000F09AFB041BA54203D8751C2E460446CE
:103D4000F3E70A2E04D9BDE87040012000F0E4BB7F
:103D500070BD0000F8B5144B0D46D96103F1100198
:103D600041600A2A1969826038BF0A2201604860EE
:103D70001861A818144600F07BFB0A2700F074FBBA
:103D8000431BA342064606D37C1C281900F07EFB89
:103D900027463546F2E70A2F04D9BDE8F84001204E
:103DA00000F0BABBF8BD00BF384E0020F8B506469B
:103DB0000D4600F059FB0F4A134653F8107F9F42FF
:103DC00006D12A4601463046BDE8F840FFF7C2BF9B
:103DD000D169BB68441A2C1928BF2C46A34202D9CA
:103DE0002946FFF79BFF224631460348BDE8F840CD
:103DF000FFF77EBF384E0020484E002010B4C0E9C7
:103E0000032300235DF8044B4361FFF7CFBF00009D
:103E100010B5194C236998420DD0D0E90032816861
:103E200013605A609A680A449A60002303604FF056
:103E3000FF33A36110BD2346026843F8102F53607F
:103E40000022026022699A4203D1BDE8104000F0CE
:103E500017BB936881680B44936000F005FB2269EF
:103E6000E1699268441AA242E4D91144BDE81040C5
:103E7000091AFFF753BF00BF384E00202DE9F04765
:103E8000DFF8BC8008F110072C4ED8F8105000F075
:103E9000EBFAD8F81C40AA68031B9A423ED8144497
:103EA000D5E900324FF00009C8F81C4013605A6091
:103EB000C5F80090D8F81030B34201D100F0E0FA14
:103EC00089F31188D5E9033128469847302383F3D5
:103ED00011886B69002BD8D000F0C6FA6A69A0EB94
:103EE00004094A4582460DD2022000F015FB00224B
:103EF000D8F81030B34208D151462846BDE8F04703
:103F0000FFF728BF121A2244F2E712EB090938BF63
:103F10004A4629463846FFF7EBFEB5E7D8F8103099
:103F2000B34208D01444211AC8F81C00A960BDE8A7
:103F3000F047FFF7F3BEBDE8F08700BF484E002012
:103F4000384E002038B500F08FFA054AD2E908450E
:103F5000031B181945F10001C2E9080138BD00BF73
:103F6000384E002000207047FEE700007047000038
:103F70004FF0FF3070470000BFF34F8F024A1369C4
:103F8000DB03FCD4704700BF0020024008B5094B9A
:103F90001B7873B9FFF7F0FF074B5A69002ABFBFC0
:103FA000064A9A6002F188329A601A6822F48062A6
:103FB0001A6008BDB8500020002002402301674568
:103FC00008B50B4B1B7893B9FFF7D6FF094B5A691D
:103FD00042F000425A611A6842F480521A601A682C
:103FE00022F480521A601A6842F480621A6008BD96
:103FF000B8500020002002407F289ABF00F5803092
:10400000C0020020704700004FF4006070470000BD
:10401000802070477F2808B50BD8FFF7EDFF00F52B
:1040200000630268013204D104308342F9D10120D7
:1040300008BD0020FCE700007F2810B504461FD80B
:10404000FFF79AFFFFF7A2FF0E4BF3221A6102223D
:104050005A615A6942EAC0025A615A6942F480328E
:104060005A61FFF789FF4FF40061FFF7C5FF00F0C9
:1040700043F9FFF7A5FF2046BDE81040FFF7CABF90
:10408000002010BD002002402DE9F84340EA020361
:1040900013F00703144606D0304B40F241321A6049
:1040A0000020BDE8F88385182D4A95420CD92B4A8B
:1040B00040F246311160F3E7031D1B684A689342E2
:1040C00008D1083C08300831072C14D902680B6865
:1040D0009A42F1D0FFF75AFFFFF74EFF214E083109
:1040E0004FF001084FF00009012CA1F1080706D894
:1040F000FFF766FF01E0002CECD10120D1E7C6F804
:104100001480054651F8083C45F8043B51F8043C3E
:104110004360FFF731FF336943F001033361C6F8B1
:104120001490026851F8083C9A420CD00B4B40F2B4
:104130006E321A600C4B18600C4B1C600C4B1F60ED
:10414000FFF73EFFACE72D6851F8043C9D4201F1BA
:104150000801EBD1083C0830C6E700BFB45000208E
:104160000000040800200240A8500020B0500020A9
:10417000AC500020084908B50B7828B11BB9FFF7EF
:1041800005FF01230B7008BD002BFCD0BDE80840E3
:104190000870FFF715BF00BFB850002008B50649EA
:1041A000064800F0ABF8BDE808404FF480414FF0FE
:1041B000805000F0A3B800BF007F01000001002084
:1041C000084600F035BA000038B5EFF311859DB907
:1041D000EFF30584C4F30804302334B183F311886A
:1041E000FFF7B0FE85F3118838BD83F31188FFF720
:1041F000A9FE84F3118838BDBDE83840FFF7A2BEA0
:1042000038B5FFF7E1FF114C114AC00840EA417090
:10421000A0FB025EC908A0FB040C1CEB050CA1FB73
:1042200004404FF000035B41A1FB02121CEB040CA5
:1042300043EB000011EB0E0142F10002411842F184
:104240000000090941EA007038BD00BFCFF753E311
:10425000A59BC4200244D2B2904200D17047431CB7
:10426000800000F1804000F51450006841F8040B14
:10427000D8B2F1E7124B10B5D3F89040240409D41A
:10428000D3F89040C3F89040D3F8904044F40044F1
:10429000C3F890400B4C2368024443F480732360BE
:1042A000D2B2904200D110BD431C800000F180408A
:1042B00000F5145051F8044B0460D8B2F1E700BF88
:1042C000001002400070004007B5012201A9002043
:1042D000FFF7C0FF019803B05DF804FB13B5044677
:1042E000FFF7F2FFA04205D0012201A900200194AE
:1042F000FFF7C0FF02B010BD70470000704700001C
:1043000070470000074B45F255521A6002225A606E
:1043100040F6FF729A604CF6CC421A60024B0122C2
:104320001A70704700300040C0500020034B1B78CB
:104330001BB1034B4AF6AA221A607047C0500020F6
:1043400000300040054B1A6832B902F1804202F594
:104350000432D2F894201A60704700BFBC5000208D
:10436000024B4FF40002C3F8942070470010024043
:1043700008B5FFF7E7FF024B1868C0F3407008BDAF
:10438000BC50002070470000FEE700000A4B0B48BD
:104390000B4A90420BD30B4BDA1C121AC11E22F0AF
:1043A00003028B4238BF00220021FCF761BE53F8A4
:1043B000041B40F8041BECE714490008445100209A
:1043C00044510020445100200023054A194601337E
:1043D000102BC2E9001102F10802F8D1704700BFAA
:1043E000C450002008B5124B9A6D42F001029A6544
:1043F0009A6F42F001029A670E4A9B6F936843F0EE
:10440000010393600620FFF74FFA0B4BB0FBF3F06C
:104410004FF080434FF0FF3201389862DA62002299
:104420009A615A63DA605A6001225A611A6008BDC3
:1044300000100240002004E040420F004FF0804294
:1044400008B51169D3680B40D9B2C9439B07116104
:1044500007D5302383F31188FFF7FEFB002383F396
:10446000118808BDFFF7BEBF4FF08043586A704700
:104470004FF08043002258631A610222DA607047CD
:104480004FF080430022DA60704700004FF0804315
:1044900058637047FEE7000070B51B4B01630025B1
:1044A000044686B0586085620E46FFF799F804F11D
:1044B0001003C4E904334FF0FF33C4E90635C4E9FF
:1044C0000044A560E562FFF7CFFF2B460246C4E932
:1044D000082304F134010D4A256580232046FFF7A7
:1044E000BDFB0123E0600A4A0375009272680192E5
:1044F000B268CDE90223074B6846CDE90435FFF7E2
:10450000D5FB06B070BD00BFA0500020A04700083A
:10451000A547000895440008024AD36A1843D062B0
:10452000704700BF384E00204B6843608B68836043
:10453000CB68C3600B6943614B6903628B6943625B
:104540000B6803607047000008B5204BDA6A42F040
:104550007F02DA62DA6A22F07F02DA62DA6ADA6C01
:1045600042F07F02DA64DA6E42F07F02DA66184ABD
:10457000DB6E11464FF09040FFF7D6FF02F11C01B1
:1045800000F58060FFF7D0FF02F1380100F5806090
:10459000FFF7CAFF02F1540100F58060FFF7C4FF86
:1045A00002F1700100F58060FFF7BEFF02F18C019F
:1045B00000F58060FFF7B8FF02F1A80100F5806008
:1045C000FFF7B2FFBDE80840FFF7F0B80010024067
:1045D000AC47000808B500F009F8FFF717FBBDE885
:1045E0000840FFF7AFBE00007047000008B5FFF7B6
:1045F000D5F8FFF7E9FEFFF7F7FFBDE80840FFF742
:1046000031BF00000B460146184600F003B8000019
:1046100000F00EB810B5054C13462CB10A46014601
:104620000220AFF3008010BD2046FCE70000000030
:10463000024B01461868FFF7C3BD00BF40230020AE
:1046400010B501390244904201D1002005E0037801
:1046500011F8014FA34201D0181B10BD0130F2E741
:104660002DE9F041A3B1C91A17780144044603F1BA
:10467000FF3C8C42204601D9002009E00578BD426C
:1046800004F10104F5D10CEB0405D618A54201D1C3
:10469000BDE8F08115F8018D16F801EDF045F5D073
:1046A000E7E70000034611F8012B03F8012B002A6D
:1046B000F9D17047696E2E736965727261616572B6
:1046C0006F73706163652E547275654E61765072BA
:1046D0006F2D47340000000040A2E4F164689106A9
:1046E0000041A3E5F2656992070000004261642081
:1046F00043414E496661636520696E6465782E00AA
:104700000000000000000000AD1D00086518000852
:10471000C1240008D518000819190008011B000859
:10472000E11800089D180008A11800087918000871
:1047300061180008BD1A000885180008F92500084E
:1047400091180008911A000801040E05054B020299
:104750000E05054B04010E05054B05010B04044B2A
:104760000801060303460000636C6B737763000067
:104770000003000000000000000100000000010133
:1047800003000000132831010407040001000000A9
:104790006330000090470008904E0020A050002099
:1047A0006D61696E0069646C650000001001942AF7
:1047B000000000009AAAAAAA00001424FBFF00002F
:1047C000000000000090090000040000000000004C
:1047D000AAA6AAAA00000000DFFF00000000000057
:1047E000000000000000000000000000AAAAAAAA21
:1047F00000000000FFFF00000000000000000000BB
:104800000000000000000000AAAAAAAA0000000000
:10481000FFFF00000000000000000000000000009A
:1048200000000000AAAAAAAA00000000FFFF0000E2
:104830000000000000000000000000000000000078
:10484000AAAAAAAA00000000FFFF000000000000C2
:10485000000000000000000000000000AAAAAAAAB0
:1048600000000000FFFF000000000000000000004A
:10487000B5140000000000000070030000000000FC
:10488000FE2A0100D2040000006889096D8BB9027C
:1048900000B4C404006889090068890900688909AE
:1048A000006889090068890900688909000000001A
:1048B0004423002000000000000000000000000071
:1048C00000000000000000000000000000000000E8
:1048D00000000000000000000000000000000000D8
:1048E00000000000000000000000000000000000C8
:1048F00000000000000000000000000000000000B8
:1049000000000000000000000000000000000000A7
:0449100000000000A3
:00000001FF
